:100000000C9462000C94C7030C94A0030C948A0017
:100010000C948A000C948A000C948A000C948A0038
:100020000C948A000C948A000C948A000C948A0028
:100030000C948A000C948A000C948A000C948A0018
:100040000C9456030C948A000C948A000C948A0039
:100050000C948A000C948A000C948A000C948A00F8
:100060000C9421050C948A00000000002300260057
:10007000290000000008000201000003040700003E
:1000800000000000000000000000250028002B00F8
:1000900000000000240027002A00040404040404D3
:1000A0000404020202020202030303030303010227
:1000B00004081020408001020408102001020408F6
:1000C0001020620911241FBECFEFD8E0DEBFCDBFE4
:1000D00011E0A0E0B1E0E4E5F1E202C005900D928C
:1000E000AC35B107D9F722E0ACE5B1E001C01D9213
:1000F000AB38B207E1F710E0C2E6D0E004C02197C8
:10010000FE010E948310C136D107C9F70E949109F0
:100110000C94A8100C94000090E0FC01E255FF4FF5
:100120002491FC01E656FF4F8491882399F090E0DA
:10013000880F991FFC01E057FF4FA591B491FC0176
:10014000EA57FF4F859194918FB7F894EC91E22B89
:10015000EC938FBF089580E480937C0080917A00B7
:10016000806480937A0080917A0086FDFCCF809134
:1001700078002091790090E0922B0895CF92DF9241
:10018000EF92FF920F931F93CF93DF936C017A014D
:100190008B01C0E0D0E0CE15DF0589F0D8016D916C
:1001A0008D01D601ED91FC910190F081E02DC60109
:1001B0000995892B11F47E0102C02196ECCFC7016D
:1001C000DF91CF911F910F91FF90EF90DF90CF9033
:1001D0000895833081F028F4813099F08230A1F0C5
:1001E00008958730A9F08830B9F08430D1F4809137
:1001F00080008F7D03C0809180008F778093800086
:10020000089584B58F7702C084B58F7D84BD08952D
:100210008091B0008F7703C08091B0008F7D809374
:10022000B00008953FB7F89480917A0190917B01D6
:10023000A0917C01B0917D0126B5A89B05C02F3F00
:1002400019F00196A11DB11D3FBFBA2FA92F982FFC
:100250008827820F911DA11DB11DBC01CD0142E077
:10026000660F771F881F991F4A95D1F708958F92BF
:100270009F92AF92BF92CF92DF92EF92FF926B016B
:100280007C010E9412014B015C01C114D104E10404
:10029000F104F1F00E941201DC01CB0188199909E7
:1002A000AA09BB09883E9340A105B10570F321E07E
:1002B000C21AD108E108F10888EE880E83E0981E82
:1002C000A11CB11CC114D104E104F10419F7DDCF64
:1002D000FF90EF90DF90CF90BF90AF909F908F9066
:1002E00008950895009769F0FC0101900020E9F756
:1002F0003197AF01481B590BBC018DE591E00C947F
:10030000BE0080E090E008958F929F92AF92BF92DE
:100310000F931F93CF93DF93CDB7DEB7A1970FB69F
:10032000F894DEBF0FBECDBF19A2423008F44AE0F8
:100330008E010F5D1F4F842E912CA12CB12CA50195
:1003400094010E943A10E62FB901CA010150110927
:10035000EA3014F4E05D01C0E95CD801EC93232B92
:10036000242B252B61F7C8010E947201A1960FB6BC
:10037000F894DEBF0FBECDBFDF91CF911F910F91DB
:10038000BF90AF909F908F900895CF92DF92EF92A1
:10039000FF92CF93DF936C01990FEE08FF08F7FEF1
:1003A0001FC0E0915D01F0915E010190F081E02DB0
:1003B0006DE28DE591E00995EC0166277727CB0189
:1003C0006C197D098E099F094AE00E9484018C0FF7
:1003D0009D1FDF91CF91FF90EF90DF90CF90089518
:1003E0004AE0C701B601DF91CF91FF90EF90DF9017
:1003F000CF900C9484010E94A310682F70E080E0DD
:1004000090E04AE00C9484010C947201643008F08E
:1004100063E090917001691710F06FEF690FE62F9C
:10042000F0E0E35AFE4F9489682F690F60688DE50C
:1004300091E00C941E05CF93DF93282F30E0F90153
:10044000EE58FF4F8491F901E255FF4FD491F90125
:10045000E656FF4FC491CC2391F081110E94E90030
:10046000EC2FF0E0EE0FFF1FE859FF4FA591B4917C
:10047000EC91ED2381E090E021F480E002C080E087
:1004800090E0DF91CF9108951F93CF93DF93282FB2
:1004900030E0F901EE58FF4F8491F901E255FF4F2A
:1004A000D491F901E656FF4FC491CC23C9F0162F21
:1004B00081110E94E900EC2FF0E0EE0FFF1FEA57D8
:1004C000FF4FA591B4918FB7F894111105C09C917D
:1004D000ED2FE095E92302C0EC91ED2BEC938FBF5B
:1004E000DF91CF911F910895CF93DF93EC0160E0EE
:1004F0008E810E94440261E08E810E94440260E08D
:100500008E810E9444028BE891E00197F1F7DF9120
:10051000CF910895CF92DF92EF92FF920F931F93A6
:10052000CF93DF937C016C0187E0C80ED11CC0E043
:10053000D0E0062F10E0B8010C2E02C0759567952B
:100540000A94E2F76170F60181916F010E94440202
:100550002196C430D10579F7C701DF91CF911F9162
:100560000F91FF90EF90DF90CF900C947402EF9278
:10057000FF920F931F93CF93DF93EC01623018F03B
:100580008F8588608F876B8B1C8A80E48D8B80E1E0
:100590008E8B80E58F8B8C810E948C008D818F3FAC
:1005A00011F00E948C008E810E948C007E0187E0F9
:1005B000E80EF11C00E010E08F8584FD03C084E0AC
:1005C00090E002C088E090E00817190744F4F701B2
:1005D00081917F010E948C000F5F1F4FEDCF8BE355
:1005E0009DE00197F1F760E08C810E94440260E099
:1005F0008E810E9444028D818F3F19F060E00E943D
:1006000044026F8564FD1DC063E0CE010E948A0232
:100610000BE416E4C8010197F1F763E0CE010E94F4
:100620008A02C8010197F1F763E0CE010E948A02B5
:1006300083E592E00197F1F762E0CE010E948A0221
:1006400016C06062CE010E941E058BE496E40197FD
:10065000F1F76F856062CE010E941E0583E592E08E
:100660000197F1F76F856062CE010E941E056F85CC
:100670006062CE010E941E0584E0888B6CE0CE0192
:100680000E941E0561E0CE010E941E058BE39FE1E2
:100690000197F1F782E0898B66E0CE01DF91CF917F
:1006A0001F910F91FF90EF900C941E051F920F92D7
:1006B0000FB60F9211242F933F938F939F93AF9375
:1006C000BF938091760190917701A0917801B091CC
:1006D00079013091750123E0230F2D3720F4019625
:1006E000A11DB11D05C026E8230F0296A11DB11D55
:1006F000209375018093760190937701A093780100
:10070000B093790180917A0190917B01A0917C0155
:10071000B0917D010196A11DB11D80937A01909346
:100720007B01A0937C01B0937D01BF91AF919F911C
:100730008F913F912F910F900FBE0F901F901895A2
:100740001F920F920FB60F9211242F933F934F9346
:100750005F936F937F938F939F93AF93BF93EF9329
:10076000FF93E0910201F09103010995FF91EF9150
:10077000BF91AF919F918F917F916F915F914F91B9
:100780003F912F910F900FBE0F901F9018951F92C1
:100790000F920FB60F9211242F933F934F935F93B5
:1007A0006F937F938F939F93AF93BF93EF93FF9339
:1007B000E0910001F09101010995FF91EF91BF9146
:1007C000AF919F918F917F916F915F914F913F91E9
:1007D0002F910F900FBE0F901F901895CF92DF9220
:1007E000EF92FF920F931F93CF93DF93EC01F62EBE
:1007F000642F8C810E9444028D818F3F19F060E04C
:100800000E9444028F850F2D10E084FF25C06E01E9
:1008100087E0C80ED11CE12CF12CB8010E2C02C0CF
:10082000759567950A94E2F76170F60181916F0101
:100830000E944402FFEFEF1AFF0A88E0E816F10475
:1008400061F7CE01DF91CF911F910F91FF90EF9053
:10085000DF90CF900C947402B80184E07595679591
:100860008A95E1F7CE010E948A026F2DCE01DF91B9
:10087000CF911F910F91FF90EF90DF90CF900C944C
:100880008A0285ED8093BC008091BC0084FDFCCF82
:1008900010926502089540913F02262F30E0240F08
:1008A000311D21323105DCF4209165022430C9F478
:1008B000FC0180E090E0861758F430913F022191CE
:1008C000DC01A35EBD4FA30FB11D2C930196F3CFA6
:1008D00080913F02680F60933F0280E0089581E0BD
:1008E000089582E0089508958FEF9FEF08958FEFA8
:1008F0009FEF089580911C0290E091958195910958
:100900000895CF93DF9300D0CDB7DEB7CB01642F2E
:1009100049835A830E944B044981842F5A81952F21
:100920000F900F90DF91CF910895CF93DF931F9297
:10093000CDB7DEB7698361E0CE0101960E944B041A
:1009400081E090E00F90DF91CF910895089580E0CD
:1009500090E008958EBD00000DB407FEFDCF8EB56A
:10096000089541E00E94EE0381E090E008954F92E7
:100970005F926F927F928F929F92AF92BF92CF922F
:10098000DF92EF92FF92880F991F880F991FFC0149
:10099000E851FE4FC080D180E280F3808D2C9E2CE8
:1009A000AF2CBB2427016624772460E082E10E94FB
:1009B0004402E3E2F0E03197F1F78F2D0E94AA04A0
:1009C000842D0E94AA04882D0E94AA048C2D0E94C6
:1009D000AA0461E082E10E9444028FE090E0019766
:1009E000F1F760E082E1FF90EF90DF90CF90BF9051
:1009F000AF909F908F907F906F905F904F900C94EE
:100A000044020F931F93CF93DF93C3E0D1E082E0C2
:100A10000E941B028C0183E00E941B020817190729
:100A200019F4D0935C0103C082E080935C01C15053
:100A300071F7DF91CF911F910F91089540E00C94D1
:100A4000EE031F920F920FB60F9211242F933F9334
:100A50004F935F936F937F938F939F93AF93BF93C6
:100A6000EF93FF938091B900887F803609F49CC092
:100A700068F5883209F45BC090F4803109F454C001
:100A800038F4882309F4F6C0883009F44DC0F6C064
:100A9000883109F44CC0803209F45DC0EFC0803465
:100AA00009F468C048F4803309F455C0883309F06C
:100AB000E5C080936402D8C0803509F44FC0883502
:100AC00009F45DC0883409F0D9C0D6C0883909F46A
:100AD000C7C0A8F4883709F467C038F4883609F429
:100AE00063C0803709F460C0C9C0883809F4B8C051
:100AF000803909F45FC0803809F0C0C05BC0803B1A
:100B000009F486C038F4803A09F466C0883A09F4DA
:100B10007FC0B4C0803C09F4A7C0883C09F4A4C0DD
:100B2000883B09F48AC0AAC080918A0210C09091C3
:100B3000890280918802981770F5E091890281E01E
:100B40008E0F80938902F0E0E859FD4F80818093F9
:100B5000BB0085EC86C0809364028EC0E091890260
:100B600081E08E0F809389028091BB00F0E0E8590C
:100B7000FD4F808390918902809188026EC0E09140
:100B8000890281E08E0F809389028091BB00F0E0A2
:100B9000E859FD4F80838091670281116DC081E02B
:100BA0008093660284EA61C083E0809365021092BC
:100BB0006302CFCF80916302803208F051C0E09190
:100BC000630281E08E0F809363028091BB00F0E0AE
:100BD000ED5BFD4F8083BDCF85EC8093BC00109210
:100BE000650280916302803230F4E0916302F0E0AC
:100BF000ED5BFD4F10826091630270E0E091410275
:100C0000F091420283E492E009951092630236C0AB
:100C100084E0809365021092400210923F02E091BE
:100C20003D02F0913E02099580913F02811105C07D
:100C300081E080933F0210921D02E091400281E02A
:100C40008E0F80934002F0E0E35EFD4F8081809341
:100C5000BB009091400280913F02981708F479CF31
:100C600085E88093BC000AC085EC8093BC0010929C
:100C7000650204C0109264020E944104FF91EF914A
:100C8000BF91AF919F918F917F916F915F914F91A4
:100C90003F912F910F900FBE0F901F9018954F927C
:100CA0005F926F927F928F929F92AF92BF92CF92FC
:100CB000DF92EF92FF920F931F93CF93DF93CDB705
:100CC000DEB728970FB6F894DEBF0FBECDBF4B013D
:100CD0005C0120E031EE45EF55E00E945C1020936E
:100CE000E701C501B40120E836E948E950E00E9477
:100CF0005C10EAE0CE2ED12CE12CF12CCA01B90116
:100D0000A70196010E945C106093E601C501B40141
:100D100020E432E44FE050E00E945C10CA01B901C7
:100D2000A70196010E945C106093E501C501B40122
:100D300020EA36E841E050E00E945C10CA01B901A7
:100D4000A70196010E945C106093E401C501B40103
:100D500020E137E240E050E00E945C10CA01B90196
:100D6000A70196010E945C106093E301C501B401E4
:100D700028EE33E040E050E00E945C10CA01B90167
:100D8000A70196010E945C106093E201C501B401C5
:100D900024E630E040E050E00E945C10CA01B90156
:100DA000A70196010E945C106093E101C501B401A6
:100DB000A70196010E945C10162FCA01B901A70174
:100DC00096010E945C106093E0011093DF0161E0E6
:100DD00080E00E9406028BE491E00E9404021091E0
:100DE000E70161E0112359F080E00E940602812FA3
:100DF0000E94FD0188E591E00E94040203C082E0A8
:100E00000E9406028091E6010E94FD018091E501A9
:100E10000E94FD018091E4010E94FD018AE591E0BC
:100E20000E9404028091E3010E94FD018091E20191
:100E30000E94FD018091E1010E94FD0188E591E0A1
:100E40000E9404028091E0010E94FD018091DF0177
:100E50000E94FD0120910A0130910B0140910C018B
:100E600050910D0121158DEF380783E4480784E187
:100E700058070CF00EC220389EEF390791E249075F
:100E80009AE059070CF00AC22034AFEF3A07A0E10C
:100E90004A07A5E05A070CF006C2203ABFE73B0715
:100EA000B8E84B07B2E05B070CF002C2203DEFE36D
:100EB0003E07E4E44E07E1E05E070CF0FEC1283E89
:100EC000FFE13F07F2EA4F0751052CF0A0E2B0E046
:100ED00005E010E004C0A0E4B0E006E010E00E94ED
:100EE0007B100E94180F20E836E948E95BE40E9475
:100EF0006E0E6B017C010E94E00E69837A838B8306
:100F00009C838091060190910701A0910801B09106
:100F100009018D839E83AF83B887A981BA81BD0102
:100F2000BB0F880B990B0E94180F9B01AC01C701E6
:100F3000B6010E94FC0D2B013C0120E030E040E8AE
:100F40005BE40E94CD0F6B017C0120E030E0A90141
:100F50000E94C80F20E030E040E05FE387FD05C05D
:100F6000C701B6010E94FD0D04C0C701B6010E9471
:100F7000FC0D0E94E00E4B015C0120E030E0A90175
:100F8000C301B2010E94690E8823C1F16D817E8187
:100F90008F8198850E94180F9B01AC0160E876E96B
:100FA00088E99BE40E946E0E0E94E00E2B013C013A
:100FB00068EE73E080E090E0A30192010E945C1073
:100FC000821A930AA40AB50AC501B4010E94160F39
:100FD0009B01AC01C701B6010E94FC0D6B017C01B5
:100FE000C301B2010E94180F9B01AC01C701B601F9
:100FF0000E94CD0F0E94E00ECB0109C0812C912CE4
:10100000540180E090E0412C512C320143944981FD
:101010005A8124E0440F551F2A95E1F7052E000C54
:10102000660B770B60624093E8015093E90160938F
:10103000EA017093EB0134E0880C991CAA1CBB1CDC
:101040003A95D1F7BFEF8B1A9B0AAB0ABB0A809285
:10105000EC019092ED01A092EE01B092EF0144E01C
:10106000440C551C661C771C4A95D1F7E2E04E0EE5
:10107000511C611C711C092E000CAA0BBB0B52E108
:10108000880F991FAA1FBB1F5A95D1F7482A592AC2
:101090006A2A7B2A4092F0015092F1016092F2019B
:1010A0007092F30183E090E0A0E0B0E08093F4015F
:1010B0009093F501A093F601B093F70184E899E8C5
:1010C000A0E0B0E38093F8019093F901A093FA01B6
:1010D000B093FB0185E290E0A0E8B0E08093FC01D2
:1010E0009093FD01A093FE01B093FF01C801110F81
:1010F000AA0BBB0B65E1880F991FAA1FBB1F6A953E
:10110000D1F786679068A460B563809300029093DE
:101110000102A0930202B093030287EE90E0A0E0E8
:10112000B2E18093040290930502A0930602B0936B
:10113000070288E294E0ADE2B0E180930802909368
:101140000902A0930A02B0930B0289EC9CE7A4E386
:10115000B5E380930C0290930D02A0930E02B0931E
:101160000F028AEF9FE3A0ECB0E08093100290930F
:101170001102A0931202B09313028BE090E3A1E658
:10118000B0E08093140290931502A0931602B093DE
:1011900017028CE194E0A1E0B0E0809318029093F4
:1011A0001902A0931A02B0931B028CE090E00E94F7
:1011B000B7040BE017E2C8010197F1F78BE090E06C
:1011C0000E94B704C8010197F1F78AE090E00E94FD
:1011D000B704C8010197F1F789E090E00E94B704D5
:1011E000C8010197F1F788E090E00E94B704C801B8
:1011F0000197F1F787E090E00E94B704C8010197DA
:10120000F1F786E090E00E94B704C8010197F1F77A
:1012100085E090E00E94B704C8010197F1F784E0EF
:1012200090E00E94B704C8010197F1F783E090E0D5
:101230000E94B704C8010197F1F782E090E00E9494
:10124000B704C8010197F1F781E090E00E94B7046C
:10125000C8010197F1F780E090E00E94B704C8014F
:101260000197F1F728960FB6F894DEBF0FBECDBFF9
:10127000DF91CF911F910F91FF90EF90DF90CF9072
:10128000BF90AF909F908F907F906F905F904F90A6
:101290000895A1E0B0E000E010E021CEA2E0B0E0CF
:1012A00001E010E01CCEA4E0B0E002E010E017CEB8
:1012B000A8E0B0E003E010E012CEA0E1B0E004E06E
:1012C00010E00DCEE3EDF1E01382128288EE93E0A0
:1012D000A0E0B0E084839583A683B78382E191E0A8
:1012E00091838083EDE5F1E01382128284E291E044
:1012F0009183808388E084838FEF858389E0868370
:1013000084E0878385E0808786E0818787E0828725
:101310001386148615861686178661E0CF010C9415
:10132000B702CF93DF9300D000D0CDB7DEB778946B
:1013300084B5826084BD84B5816084BD85B58260DA
:1013400085BD85B5816085BD80916E00816080938B
:101350006E001092810080918100826080938100F4
:101360008091810081608093810080918000816004
:10137000809380008091B10084608093B10080915F
:10138000B00081608093B00080917A008460809387
:101390007A0080917A00826080937A0080917A004E
:1013A000816080937A0080917A00806880937A00CF
:1013B0001092C10062E08DE591E00E94B70260E00A
:1013C00080E00E9406028CE291E00E94040282E129
:1013D0000E948C0060E082E10E9444028CB5837F11
:1013E0008CBD8CB58F7D8CBD8CB583608CBD8DB56F
:1013F0008E7F8DBD1FB7F89480917E01811124C02E
:10140000E4EAF0E08491E8EBF0E09491E82FF0E07A
:10141000EE0FFF1FE057FF4FA591B491EC91E92328
:1014200021F461E08AE00E9444028AE00E948C007C
:101430008CB580618CBD8CB580648CBD8DE00E94C4
:101440008C008BE00E948C0080917E018F5F8093E6
:101450007E011FBF6CED75E080E090E00E943701D7
:1014600088EE93E0A0E0B0E0809383019093840144
:10147000A0938501B093860184EC99E0A0E0B0E0F0
:101480008093870190938801A0938901B0938A018A
:1014900080E197E2A0E0B0E080938B0190938C0113
:1014A000A0938D01B0938E0120EA36E841E050E030
:1014B00020938F01309390014093910150939201BA
:1014C00080E492E4AFE0B0E08093930190939401C4
:1014D000A0939501B093960180E896E9A8E9B0E061
:1014E0008093970190939801A0939901B0939A01EA
:1014F00060ECC62E65E6D62E62E5E62EF12CC09293
:101500009B01D0929C01E0929D01F0929E018093FC
:101510009F019093A001A093A101B093A20180E04C
:101520009AEBABEDB0E08093A3019093A401A0935C
:10153000A501B093A60180EA90E4ADEDB0E0809300
:10154000A7019093A801A093A901B093AA0180ECF0
:1015500090E2A0E9B2E08093AB019093AC01A0933C
:10156000AD01B093AE0180EE91ECA7E9B2E08093BB
:10157000AF019093B001A093B101B093B20180ECA0
:101580009AE7A2EFB4E08093B3019093B401A093E3
:10159000B501B093B60180E499E5A3E7B7E0809385
:1015A000B7019093B801A093B901B093BA0180EA52
:1015B00096E2ADEBBDE08093BB019093BC01A0939C
:1015C000BD01B093BE0180E093EAA1EEB1E180934A
:1015D000BF019093C001A093C101B093C20180E00C
:1015E0009EEDA9E3BAE18093C3019093C401A09357
:1015F000C501B093C60180E099E1A2E9B2E280930F
:10160000C7019093C801A093C901B093CA0180E0BB
:101610009AEFA7E8B8E28093CB019093CC01A09316
:10162000CD01B093CE0160E080E029833A834B8303
:101630005C830E9406028FE491E00E94040260E055
:1016400080E00E9406028DE391E00E940402609116
:10165000060170910701809108019091090129818B
:101660003A814B815C810E945C103093820120930F
:101670008101C9010E94C50183E491E00E94040236
:1016800061E08CE00E94060282E491E00E94040284
:1016900060910A0170910B0180910C0190910D01F4
:1016A0000E944F0661E082E00E94440261E083E014
:1016B0000E94440281E095E0909301018093000133
:1016C000809169008C7F816080936900E89A812C09
:1016D0007AEF972E77E8A72E78E2B72EE0EC4E2E21
:1016E000E5E65E2EE2E56E2E712C30E0232E30E032
:1016F000332E80915C018130C9F540910A015091EF
:101700000B0160910C0170910D0180910601909187
:101710000701A0910801B0910901840F951FA61F30
:10172000B71F81300AEF900707E8A00708E2B0076B
:101730004CF480930A0190930B01A0930C01B09399
:101740000D0108C080920A0190920B01A0920C0139
:10175000B0920D0160910A0170910B0180910C0112
:1017600090910D010E944F0610925C0180915C01E6
:101770008230C1F580910A0190910B01A0910C017A
:10178000B0910D014091060150910701609108014F
:1017900070910901841B950BA60BB70B803C15E6D5
:1017A000910712E5A107B1054CF080930A019093CF
:1017B0000B01A0930C01B0930D0108C040920A01E7
:1017C00050920B0160920C0170920D0160910A0120
:1017D00070910B0180910C0190910D010E944F06B8
:1017E00010925C010E94AB009093800180937F0176
:1017F000893E23E092078CF4823391058CF0833C80
:1018000091058CF08C3731E0930784F08B3202E045
:1018100090077CF0863193407CF085E090E00EC02C
:1018200080E090E00BC081E090E008C082E090E0B2
:1018300005C083E090E002C084E090E09093D20184
:101840008093D1018230910509F46CC1F4F40097C2
:1018500021F1019709F0B6C140910A0150910B01A5
:1018600060910C0170910D0180910601909107012A
:10187000A0910801B09109018A019B01080F191F6D
:101880002A1F3B1FC901B80163C18330910509F4C8
:10189000DDC0049709F467C195C1E091CF01F091D3
:1018A000D001EE0FFF1FEE0FFF1FE556FE4F4081E8
:1018B00051816281738140930A0150930B016093BF
:1018C0000C0170930D018091060190910701A09188
:1018D0000801B09109016A017B01803A26E892076C
:1018E00021E0A207B10541F430E8C30E36E9D31E6A
:1018F00038E9E31EF11C23C0803402E490070FE0B6
:10190000A007B10549F410E8C11A1FE0D10A15E09B
:10191000E10A1DEFF10A13C080389649A849B105C4
:1019200039F43FE1D31A3AE0E30A3AEFF30A07C089
:1019300080E4C80E8DE0D81E83E0E81EF11C809183
:101940000A0190910B01A0910C01B0910D01409101
:1019500006015091070160910801709109018C15F1
:101960009D05AE05BF059CF48C019D01040F151F5C
:10197000261F371FC901B80100930A0110930B01FC
:1019800020930C0130930D010E944F06D8CF403AAE
:1019900016E8510711E06107710541F420E8C21A09
:1019A00026E9D20A28E9E20AF10827C0403432E4E5
:1019B00053073FE06307710559F46C017D0100E8AE
:1019C000C01A00EFD00A0AEFE00A02E0F00A15C0E0
:1019D000403856496849710549F46C017D0121EE92
:1019E000D21A25EFE20A25E0F20A07C030E4C31A52
:1019F0003DE0D30A33E0E30AF10880910A019091B7
:101A00000B01A0910C01B0910D01C816D906EA0690
:101A1000FB060CF0D7C04091060150910701609180
:101A20000801709109018C019D01041B150B260B07
:101A3000370BC901B80100930A0110930B012093E1
:101A40000C0130930D010E944F06D7CF8091040105
:101A5000909105010196863091052CF49093050133
:101A60008093040104C01092050110920401E091DA
:101A70000401F0910501EE0FFF1FEE0FFF1FED5760
:101A8000FE4F80819181A281B38180930601909362
:101A90000701A0930801B093090160E084E00E946F
:101AA000060280E591E00E94040260E084E00E946A
:101AB00006026091060170910701809108019091E2
:101AC0000901603A16E8710711E08107910584F475
:101AD00024E630E040E050E00E945C103093820148
:101AE00020938101C9010E94C50187E491E00FC0E4
:101AF00020EA36E841E050E00E945C103093820119
:101B000020938101C9010E94C50183E491E00E94F4
:101B1000040260910A0170910B0180910C01909177
:101B20000D0148C080910A0190910B01A0910C0118
:101B3000B0910D010091060110910701209108015B
:101B400030910901BC01CD01601B710B820B930B1D
:101B500060930A0170930B0180930C0190930D0127
:101B60000E944F062FC08091CF019091D001019625
:101B70008D3091052CF49093D0018093CF0104C057
:101B80001092D0011092CF01E091CF01F091D001DD
:101B9000EE0FFF1FEE0FFF1FE556FE4F60817181B4
:101BA0008281938160930A0170930B0180930C01F1
:101BB00090930D010E944F0668EC70E080E090E089
:101BC0000E9437010E94AB009093800180937F01B7
:101BD00064E170E080E090E00E94370180917F0135
:101BE00090918001843893406CF32114310409F4FE
:101BF00080CD0E94000079CD5058BB27AA270E94B3
:101C0000140E0C948E0F0E94800F38F00E94870FE4
:101C100020F039F49F3F19F426F40C947D0F0EF454
:101C2000E095E7FB0C94770FE92F0E949F0F58F384
:101C3000BA17620773078407950720F079F4A6F5B1
:101C40000C94C10F0EF4E0950B2EBA2FA02D0B01B2
:101C5000B90190010C01CA01A0011124FF27591BF1
:101C600099F0593F50F4503E68F11A16F040A22FF7
:101C7000232F342F4427585FF3CF46953795279568
:101C8000A795F0405395C9F77EF41F16BA0B620B67
:101C9000730B840BBAF09150A1F0FF0FBB1F661FAE
:101CA000771F881FC2F70EC0BA0F621F731F841FF1
:101CB00048F4879577956795B795F7959E3F08F017
:101CC000B0CF9395880F08F09927EE0F97958795D9
:101CD00008950E94530F08F481E008950E94820E37
:101CE0000C948E0F0E94870F58F00E94800F40F0D6
:101CF00029F45F3F29F00C94770F51110C94C20F17
:101D00000C947D0F0E949F0F68F39923B1F3552324
:101D100091F3951B550BBB27AA27621773078407FE
:101D200038F09F5F5F4F220F331F441FAA1FA9F394
:101D300035D00E2E3AF0E0E832D091505040E69582
:101D4000001CCAF72BD0FE2F29D0660F771F881FE3
:101D5000BB1F261737074807AB07B0E809F0BB0BD6
:101D6000802DBF01FF2793585F4F3AF09E3F5105EA
:101D700078F00C94770F0C94C20F5F3FE4F3983E19
:101D8000D4F3869577956795B795F7959F5FC9F7D3
:101D9000880F911D9695879597F90895E1E0660F54
:101DA000771F881FBB1F621773078407BA0720F0CD
:101DB000621B730B840BBA0BEE1F88F7E095089536
:101DC0000E94E70E6894B1110C94C20F08950E940E
:101DD000A70F88F09F5798F0B92F9927B751B0F007
:101DE000E1F0660F771F881F991F1AF0BA95C9F79F
:101DF00014C0B13091F00E94C10FB1E008950C946D
:101E0000C10F672F782F8827B85F39F0B93FCCF31F
:101E1000869577956795B395D9F73EF4909580951B
:101E2000709561957F4F8F4F9F4F0895E89409C03B
:101E300097FB3EF490958095709561957F4F8F4FFD
:101E40009F4F9923A9F0F92F96E9BB279395F69513
:101E5000879577956795B795F111F8CFFAF4BB0F91
:101E600011F460FF1BC06F5F7F4F8F4F9F4F16C0F5
:101E7000882311F096E911C0772321F09EE8872F7F
:101E8000762F05C0662371F096E8862F70E060E03B
:101E90002AF09A95660F771F881FDAF7880F9695B4
:101EA000879597F90895990F0008550FAA0BE0E858
:101EB000FEEF16161706E807F907C0F0121613060C
:101EC000E407F50798F0621B730B840B950B39F44C
:101ED0000A2661F0232B242B252B21F408950A26B2
:101EE00009F4A140A6958FEF811D811D089597F9F2
:101EF0009F6780E870E060E008959FEF80EC0895B0
:101F000000240A94161617061806090608950024D8
:101F10000A9412161306140605060895092E039452
:101F2000000C11F4882352F0BB0F40F4BF2B11F4C6
:101F300060FF04C06F5F7F4F8F4F9F4F089557FD25
:101F40009058440F551F59F05F3F71F04795880F27
:101F500097FB991F61F09F3F79F0879508951216BE
:101F600013061406551FF2CF4695F1DF08C016166A
:101F700017061806991FF1CF86957105610508941B
:101F80000895E894BB2766277727CB0197F9089532
:101F90000E94530F08F48FEF08950E94E00F0C94F5
:101FA0008E0F0E94800F38F00E94870F20F095233B
:101FB00011F00C94770F0C947D0F11240C94C20F28
:101FC0000E949F0F70F3959FC1F3950F50E0551F2E
:101FD000629FF001729FBB27F00DB11D639FAA277E
:101FE000F00DB11DAA1F649F6627B00DA11D661FCD
:101FF000829F2227B00DA11D621F739FB00DA11DEE
:10200000621F839FA00D611D221F749F3327A00DA7
:10201000611D231F849F600D211D822F762F6A2F43
:1020200011249F5750409AF0F1F088234AF0EE0FA8
:10203000FF1FBB1F661F771F881F91505040A9F7D5
:102040009E3F510580F00C94770F0C94C20F5F3FB8
:10205000E4F3983ED4F3869577956795B795F79511
:10206000E7959F5FC1F7FE2B880F911D9695879589
:1020700097F90895A1E21A2EAA1BBB1BFD010DC002
:10208000AA1FBB1FEE1FFF1FA217B307E407F50728
:1020900020F0A21BB30BE40BF50B661F771F881F04
:1020A000991F1A9469F760957095809590959B019A
:1020B000AC01BD01CF010895052E97FB1EF40094DD
:1020C0000E94731057FD07D00E943A1007FC03D0FE
:1020D0004EF40C94731050954095309521953F4FD8
:1020E0004F4F5F4F089590958095709561957F4F04
:1020F0008F4F9F4F0895B7FF0C9489100E9489104D
:10210000821B930B0895EE0FFF1F0590F491E02DB5
:1021100009940E949410A59F900DB49F900DA49FC8
:10212000800D911D11240895A29FB001B39FC0019D
:10213000A39F700D811D1124911DB29F700D811DF3
:102140001124911D089581E090E0F8940C94A8105A
:04215000F894FFCF31
:10215400710171010300A08601008093DC1400006A
:10216400000095048104A70473047A0477047404BA
:1021740000000000B104BE00A704A60420414446A8
:10218400353335352020204634464457005061739A
:102194003D00204D687A004B687A002020202020E2
:0C21A40020202020202020002E002C00F5
:00000001FF
